:1000000010C01FC01EC01DC01CC01BC01AC019C01C
:1000100018C017C016C015C014C013C012C011C03C
:1000200010C011241FBECFE5D1E0DEBFCDBF21E05F
:10003000A0E0B1E001C01D92A130B207E1F777D096
:10004000F7C0DECF0F931F9300E010E09801061772
:1000500017072807390759F0EFECF7E03197F1F768
:1000600000C000000F5F1F4F2F4F3F4FF0CF1F9179
:100070000F9108953F924F929BB3907F9BBB9DE160
:100080009A95F1F7000020E8422E942D4420A9F023
:10009000962359F09BB39F609BBB469400000000E1
:1000A00000009BB3907F9BBBF0CF9BB39F609BBB3B
:1000B0009BB3907F9BBB4694E8CF90E8492E942D4C
:1000C0004420A9F0982359F09BB39F609BBB4694B2
:1000D0000000000000009BB3907F9BBBF0CF9BB360
:1000E0009F609BBB9BB3907F9BBB4694E8CF80E80F
:1000F000482E842D4420A9F0842359F08BB38F60BF
:100100008BBB46940000000000008BB3807F8BBB4C
:10011000F0CF8BB38F608BBB8BB3807F8BBB469450
:10012000E8CF8BB38F608BBB4F903F9008958FECDF
:1001300097E00197F1F700C00000F89417BA83E048
:100140008093620088BB8AB38F608ABB8BB38F6059
:100150008BBB8FEC97E00197F1F700C0000040E106
:1001600060E180E187DF8FE19EE40197F1F700C055
:10017000000040E160E180E17DDF8091B2008064B9
:100180008093B200D59A90E0C0E1D0E110E1809177
:10019000B10087FFFCCF8091B000809300011092E6
:1001A000B0008091B10080688093B100809100011F
:1001B0008F3F11F4D59813C0809100018E3F89F4D0
:1001C000D5984C2F6D2F812F55DF8FE19EE401973D
:1001D000F1F700C000004C2F6D2F812F4BDF90E016
:1001E000D6CF9230E9F038F4992369F0913079F65E
:1001F000D59892E0CCCF9330B9F0943041F6C091CD
:10020000000195E0C4CF80910001813011F09FEF93
:10021000BECFD59A86B3806A8093B00091E0B7CF05
:100220001091000193E0B3CFD091000194E0AFCFE3
:04023000F894FFCF70
:00000001FF
